:020000040000FA
:100000000C945D000C9485000C9485000C94850084
:100010000C9485000C9485000C9485000C9485004C
:100020000C9485000C9485000C9485000C9485003C
:100030000C9485000C9485000C9485000C9485002C
:100040000C948A030C9485000C9458030C9432038E
:100050000C9485000C9485000C9485000C9485000C
:100060000C9485000C94850000000008000201003B
:100070000003040700000000000000000000000072
:10008000250028002B0000000000240027002A0083
:10009000040404040404040402020202020203032E
:1000A0000303030301020408102040800102040836
:1000B00010200102040810204F0511241FBECFEFAD
:1000C000D8E0DEBFCDBF11E0A0E0B1E0E4ECFFE09E
:1000D00002C005900D92A834B107D9F721E0A8E439
:1000E000B1E001C01D92AE3EB207E1F710E0CDE5F0
:1000F000D0E004C02197FE010E94DA07CC35D10779
:10010000C9F70E94D4030C94E0070C940000AF924E
:10011000BF92CF92DF92EF92FF920F931F93CF93F4
:10012000DF936C017B018B01040F151FEB015E0156
:10013000AE18BF08C017D10759F06991D601ED91EB
:10014000FC910190F081E02DC6010995892B79F78A
:10015000C501DF91CF911F910F91FF90EF90DF903C
:10016000CF90BF90AF900895FC01538D448D252F03
:1001700030E0842F90E0821B930B541710F0CF9641
:10018000089501970895FC01918D828D981761F073
:10019000A28DAE0FBF2FB11D5D968C91928D9F5F8A
:1001A0009F73928F90E008958FEF9FEF0895FC0169
:1001B000918D828D981731F0828DE80FF11D858D1C
:1001C00090E008958FEF9FEF0895FC01918D228DAF
:1001D000892F90E0805C9F4F821B91098F73992734
:1001E000089581E591E00E94E50021E0892B09F462
:1001F00020E0822F089580E090E0892B29F00E9472
:10020000F10081110C9400000895FC01A48DA80F49
:10021000B92FB11DA35ABF4F2C91848D90E0019648
:100220008F739927848FA689B7892C93A089B18968
:100230008C91837080648C93938D848D981306C009
:100240000288F389E02D80818F7D80830895EF926D
:10025000FF920F931F93CF93DF93EC0181E0888F80
:100260009B8D8C8D98131AC0E889F989808185FF50
:1002700015C09FB7F894EE89FF896083E889F989F2
:1002800080818370806480839FBF81E090E0DF91F4
:10029000CF911F910F91FF90EF900895F62E0B8D47
:1002A00010E00F5F1F4F0F731127E02E8C8D8E1102
:1002B0000CC00FB607FCFACFE889F989808185FF69
:1002C000F5CFCE010E940501F1CFEB8DEC0FFD2F94
:1002D000F11DE35AFF4FF0829FB7F8940B8FEA8924
:1002E000FB8980818062CFCFCF93DF93EC01888D33
:1002F0008823B9F0AA89BB89E889F9898C9185FDA1
:1003000003C0808186FD0DC00FB607FCF7CF8C912E
:1003100085FFF2CF808185FFEDCFCE010E940501E0
:10032000E9CFDF91CF91089590E0FC01E859FF4FAC
:100330002491FC01EC55FF4F3491FC01E057FF4F35
:10034000E491EE23C9F0222339F0233001F1A8F41F
:10035000213019F1223029F1F0E0EE0FFF1FE458AF
:10036000FF4FA591B4918FB7F894EC91611126C01D
:1003700030953E233C938FBF08952730A9F0283055
:10038000C9F0243049F7809180008F7D03C08091AF
:1003900080008F7780938000DFCF84B58F7784BD16
:1003A000DBCF84B58F7DFBCF8091B0008F778093BA
:1003B000B000D2CF8091B0008F7DF9CF3E2BDACF45
:1003C0003FB7F89480914D0190914E01A0914F015B
:1003D000B091500126B5A89B05C02F3F19F001969A
:1003E000A11DB11D3FBFBA2FA92F982F8827BC018F
:1003F000CD01620F711D811D911D42E0660F771FB7
:10040000881F991F4A95D1F70895FC01019000209B
:10041000E9F73197AF01481B590BBC0181E591E029
:100420000C9487008F929F92AF92BF920F931F936D
:10043000CF93DF93CDB7DEB7A1970FB6F894DEBFA9
:100440000FBECDBF19A2423008F44AE08E010F5D05
:100450001F4F842E912CB12CA12CA50194010E9438
:10046000B807E62FB901CA01EA30F4F4E05DD8011B
:10047000EE938D01232B242B252B79F790E080E040
:10048000109719F0CD010E940502A1960FB6F894BD
:10049000DEBF0FBECDBFDF91CF911F910F91BF90F7
:1004A000AF909F908F900895E95CE1CF4F925F925B
:1004B0006F927F928F929F92AF92BF92CF92DF9274
:1004C000EF92FF920F931F93CF936B017C01742ED9
:1004D000AC019B010E94B307882399F082E191E06F
:1004E000CF911F910F91FF90EF90DF90CF90BF9031
:1004F000AF909F908F907F906F905F904F900C94F3
:10050000050246015701E894B7F82FEF3FEF4FE798
:100510005FE7C501B4010E94B30781110DC02FEF41
:100520003FEF4FE75FE7C501B4010E94E9051816E8
:100530001CF486E191E0D4CF2FEF3FEF4FE75FE46B
:10054000C701B6010E94410718161CF48AE191E028
:10055000C7CF2FEF3FEF4FE75FECC701B6010E9417
:10056000E90587FDF3CF20E030E0A901C701B6011E
:100570000E94E90510E000E087FF0AC06DE281E516
:1005800091E00E9427018C01F7FAF094F7F8F094BB
:10059000C0E060E070E080E09FE37C1641F020E086
:1005A00030E040E251E40E94EE05CF5FF6CFA701B4
:1005B00096010E947D052B013C010E9460064B01C3
:1005C0005C014AE00E9412027C01E00EF11ECC2385
:1005D000C1F1C501B4010E948F069B01AC01C301AA
:1005E000B2010E947C054B015C016EE281E591E065
:1005F0000E942701E80EF91EC15018F120E030E0FA
:1006000040E251E4C501B4010E9446072B013C01C0
:100610000E9460064B01B12CA12C4AE0C501B40137
:100620000E941202E80EF91EC501B4010E948F0655
:100630009B01AC01C301B2010E947C054B015C012E
:10064000DBCFC701CF911F910F91FF90EF90DF900B
:10065000CF90BF90AF909F908F907F906F905F9062
:100660004F9008951F920F920FB60F9211242F935F
:100670003F934F935F936F937F938F939F93AF932A
:10068000BF93EF93FF9381E591E00E940501FF91F5
:10069000EF91BF91AF919F918F917F916F915F91FA
:1006A0004F913F912F910F900FBE0F901F90189573
:1006B0001F920F920FB60F9211242F938F939F9337
:1006C000EF93FF93E0916101F09162018081E091ED
:1006D0006701F091680182FD1BC0908180916A01E1
:1006E0008F5F8F7320916B01821741F0E0916A0157
:1006F000F0E0EF5AFE4F958F80936A01FF91EF91E2
:100700009F918F912F910F900FBE0F901F90189572
:100710008081F4CF1F920F920FB60F9211242F9366
:100720003F938F939F93AF93BF9380914901909193
:100730004A01A0914B01B0914C013091480123E056
:10074000230F2D3758F50196A11DB11D20934801A7
:100750008093490190934A01A0934B01B0934C01BF
:1007600080914D0190914E01A0914F01B0915001A7
:100770000196A11DB11D80934D0190934E01A09350
:100780004F01B0935001BF91AF919F918F913F91D5
:100790002F910F900FBE0F901F90189526E8230FF2
:1007A0000296A11DB11DD2CF789484B5826084BD1C
:1007B00084B5816084BD85B5826085BD85B5816065
:1007C00085BD80916E00816080936E0010928100E3
:1007D000809181008260809381008091810081609E
:1007E000809381008091800081608093800080915F
:1007F000B10084608093B1008091B00081608093EB
:10080000B00080917A00846080937A0080917A00B1
:10081000826080937A0080917A00816080937A0070
:1008200080917A00806880937A001092C100E091F4
:100830006101F091620182E08083E0915D01F091BD
:100840005E011082E0915F01F09160018FEC808386
:1008500010926901E0916501F091660186E0808364
:10086000E0916301F0916401808180618083E09177
:100870006301F0916401808188608083E09163016D
:10088000F0916401808180688083E0916301F09140
:10089000640180818F7D8083C2E0D0E08C2FFE01D7
:1008A000EC55FF4F9491FE01E057FF4F2491222316
:1008B00099F030E0220F331FF901EA57FF4FA5915D
:1008C000B491F901E458FF4F259134912FB7F89472
:1008D000EC91E92BEC932FBF60E00E9494012196EC
:1008E000C530D105D9F680E4B82E00E010E0B09212
:1008F0007C0080917A00806480937A0080917A00F5
:1009000086FDFCCF80917800C0917900DC2FC82F44
:100910008EE191E00E9405026E010D2E000CEE08A2
:10092000FF084AE0C701B601D7FF0DC06DE281E5BF
:1009300091E00E94270166277727CB016C197D097A
:100940008E099F094AE00E941202C701B6010E9467
:10095000910620E030E040E85AE30E94460720E09C
:1009600030E040EA50E40E9446076B017C018DE2D2
:1009700091E00E94050242E0C701B6010E945602C2
:1009800087E391E00E94050220E030E040E05FE371
:10099000C701B6010E947C0520E030E048EC52E43B
:1009A0000E9446076B017C0142E00E94560285E4EA
:1009B00091E00E94050220E030E048E851E4C701E0
:1009C000B6010E94E90560E087FD15C020E030E037
:1009D00048E851E4C701B6010E94410787FD31C0D4
:1009E00020E030E048E951E4C701B6010E94E90582
:1009F00087FF27C061E082E00E94940160E083E00D
:100A00000E94940160E084E00E9494010E94E00151
:100A10006B017C010E94E0016C197D098E099F0920
:100A2000683E734081059105A8F30115110509F48D
:100A30005ECF0E94F100882309F459CF0E94000084
:100A400056CF20E030E048E951E4C701B6010E94EA
:100A5000410787FD10C020E030E040EA51E4C701C3
:100A6000B6010E94E90587FF06C061E082E00E94AE
:100A7000940161E0C4CF20E030E040EA51E4C701D6
:100A8000B6010E94410787FDC1CF61E082E00E946C
:100A9000940161E083E00E94940161E0B4CFE1E55C
:100AA000F1E01382128288EE93E0A0E0B0E084834C
:100AB0009583A683B78384E091E09183808385EC5E
:100AC00090E09587848784EC90E09787868780EC18
:100AD00090E0918B808B81EC90E0938B828B82EC09
:100AE00090E0958B848B86EC90E0978B868B118EB3
:100AF000128E138E148E08955058BB27AA270E9479
:100B000094050C9407070E94F90638F00E9400072C
:100B100020F039F49F3F19F426F40C94F6060EF4F5
:100B2000E095E7FB0C94F006E92F0E94180758F3B4
:100B3000BA17620773078407950720F079F4A6F5C2
:100B40000C943A070EF4E0950B2EBA2FA02D0B0152
:100B5000B90190010C01CA01A0011124FF27591B02
:100B600099F0593F50F4503E68F11A16F040A22F08
:100B7000232F342F4427585FF3CF46953795279579
:100B8000A795F0405395C9F77EF41F16BA0B620B78
:100B9000730B840BBAF09150A1F0FF0FBB1F661FBF
:100BA000771F881FC2F70EC0BA0F621F731F841F02
:100BB00048F4879577956795B795F7959E3F08F028
:100BC000B0CF9395880F08F09927EE0F97958795EA
:100BD00008950E94CC0608F481E008950E94020660
:100BE0000C9407070E94000758F00E94F90640F095
:100BF00029F45F3F29F00C94F00651110C943B0747
:100C00000C94F6060E94180768F39923B1F3552354
:100C100091F3951B550BBB27AA276217730784070F
:100C200038F09F5F5F4F220F331F441FAA1FA9F3A5
:100C300035D00E2E3AF0E0E832D091505040E69593
:100C4000001CCAF72BD0FE2F29D0660F771F881FF4
:100C5000BB1F261737074807AB07B0E809F0BB0BE7
:100C6000802DBF01FF2793585F4F3AF09E3F5105FB
:100C700078F00C94F0060C943B075F3FE4F3983E49
:100C8000D4F3869577956795B795F7959F5FC9F7E4
:100C9000880F911D9695879597F90895E1E0660F65
:100CA000771F881FBB1F621773078407BA0720F0DE
:100CB000621B730B840BBA0BEE1F88F7E095089547
:100CC0000E94200788F09F5798F0B92F9927B751B5
:100CD000B0F0E1F0660F771F881F991F1AF0BA95E0
:100CE000C9F714C0B13091F00E943A07B1E00895FD
:100CF0000C943A07672F782F8827B85F39F0B93FEF
:100D0000CCF3869577956795B395D9F73EF4909592
:100D10008095709561957F4F8F4F9F4F0895E89410
:100D200009C097FB3EF490958095709561957F4F33
:100D30008F4F9F4F9923A9F0F92F96E9BB279395E1
:100D4000F695879577956795B795F111F8CFFAF4F1
:100D5000BB0F11F460FF1BC06F5F7F4F8F4F9F4F22
:100D600016C0882311F096E911C0772321F09EE880
:100D7000872F762F05C0662371F096E8862F70E0E6
:100D800060E02AF09A95660F771F881FDAF7880FC0
:100D90009695879597F90895990F0008550FAA0B16
:100DA000E0E8FEEF16161706E807F907C0F012167E
:100DB0001306E407F50798F0621B730B840B950B81
:100DC00039F40A2661F0232B242B252B21F40895D6
:100DD0000A2609F4A140A6958FEF811D811D089573
:100DE00097F99F6780E870E060E008959FEF80ECDE
:100DF000089500240A941616170618060906089581
:100E000000240A9412161306140605060895092EE6
:100E10000394000C11F4882352F0BB0F40F4BF2B55
:100E200011F460FF04C06F5F7F4F8F4F9F4F089595
:100E300057FD9058440F551F59F05F3F71F047958B
:100E4000880F97FB991F61F09F3F79F08795089570
:100E5000121613061406551FF2CF4695F1DF08C08F
:100E6000161617061806991FF1CF869571056105AC
:100E700008940895E894BB2766277727CB0197F954
:100E800008950E94CC0608F48FEF08950E94590738
:100E90000C9407070E94F90638F00E94000720F022
:100EA000952311F00C94F0060C94F60611240C9482
:100EB0003B070E94180770F3959FC1F3950F50E010
:100EC000551F629FF001729FBB27F00DB11D639FFC
:100ED000AA27F00DB11DAA1F649F6627B00DA11DA2
:100EE000661F829F2227B00DA11D621F739FB00D48
:100EF000A11D621F839FA00D611D221F749F3327B8
:100F0000A00D611D231F849F600D211D822F762F50
:100F10006A2F11249F5750409AF0F1F088234AF02D
:100F2000EE0FFF1FBB1F661F771F881F9150504099
:100F3000A9F79E3F510580F00C94F0060C943B07F6
:100F40005F3FE4F3983ED4F3869577956795B79520
:100F5000F795E7959F5FC1F7FE2B880F911D96953A
:100F6000879597F908950E94CC06880B990B0895F0
:100F7000A1E21A2EAA1BBB1BFD010DC0AA1FBB1F9D
:100F8000EE1FFF1FA217B307E407F50720F0A21B0F
:100F9000B30BE40BF50B661F771F881F991F1A947C
:100FA00069F760957095809590959B01AC01BD01A6
:100FB000CF010895EE0FFF1F0590F491E02D0994E5
:100FC000F894FFCF0000000027018700B4007401EF
:100FD000E500C300D7006E616E00696E66006F7633
:100FE000660053656E736F722076616C75653A208A
:100FF000002C20566F6C74733A20002C20646567B7
:0C1000007265657320433A20000A00006E
:107E0000112484B714BE81FFF0D085E080938100F7
:107E100082E08093C00088E18093C10086E0809377
:107E2000C20080E18093C4008EE0C9D0259A86E02C
:107E300020E33CEF91E0309385002093840096BBD3
:107E4000B09BFECF1D9AA8958150A9F7CC24DD24C4
:107E500088248394B5E0AB2EA1E19A2EF3E0BF2EE7
:107E6000A2D0813461F49FD0082FAFD0023811F036
:107E7000013811F484E001C083E08DD089C08234E0
:107E800011F484E103C0853419F485E0A6D080C0E4
:107E9000853579F488D0E82EFF2485D0082F10E0AE
:107EA000102F00270E291F29000F111F8ED06801E7
:107EB0006FC0863521F484E090D080E0DECF843638
:107EC00009F040C070D06FD0082F6DD080E0C81688
:107ED00080E7D80618F4F601B7BEE895C0E0D1E017
:107EE00062D089930C17E1F7F0E0CF16F0E7DF06D8
:107EF00018F0F601B7BEE89568D007B600FCFDCFD4
:107F0000A601A0E0B1E02C9130E011968C91119780
:107F100090E0982F8827822B932B1296FA010C0160
:107F200087BEE89511244E5F5F4FF1E0A038BF0790
:107F300051F7F601A7BEE89507B600FCFDCF97BE46
:107F4000E89526C08437B1F42ED02DD0F82E2BD052
:107F50003CD0F601EF2C8F010F5F1F4F84911BD097
:107F6000EA94F801C1F70894C11CD11CFA94CF0C13
:107F7000D11C0EC0853739F428D08EE10CD085E9AC
:107F80000AD08FE07ACF813511F488E018D01DD067
:107F900080E101D065CF982F8091C00085FFFCCF94
:107FA0009093C60008958091C00087FFFCCF809118
:107FB000C00084FD01C0A8958091C6000895E0E648
:107FC000F0E098E1908380830895EDDF803219F02E
:107FD00088E0F5DFFFCF84E1DECF1F93182FE3DFCA
:107FE0001150E9F7F2DF1F91089580E0E8DFEE27F6
:047FF000FF270994CA
:027FFE00040479
:00000001FF
